:020000040800F2
:10500000081B0020D55000084D880008C17E00080C
:105010000000000000000000000000000000000090
:105020000000000000000000000000006192000885
:105030000000000000000000699000085D93000877
:10504000E7500008E7500008E7500008E750000864
:10505000E7500008255C0008E7500008E75000080A
:1050600000000000E7500008615B0008E7500008FE
:10507000E75000083D84000800000000E7500008E9
:1050800000000000E75000080000000000000000E1
:10509000E750000800000000E7500008E750000853
:1050A000E7500008E7500008E7500008459C00085A
:1050B000E7500008E7500008000000000000000072
:1050C0000348854600F09EFC00480047ADAF00084D
:1050D000081B00200448804704480047FEE7FEE71D
:1050E000FEE7FEE7FEE7FEE7F9930008C15000087F
:1050F00030B50B46014600202022012409E00D4670
:10510000D5409D4205D31D469540491B25469540F7
:1051100040191546521E002DF1DC30BD70B500243B
:105120002546002801DA01244042002901DA012540
:105130004942FFF7DDFFAC4200D04042002C00D0D6
:10514000494270BDF0B51FB40646002082B0054646
:105150004024019100901BE0019922460F46304601
:1051600000F064FB049A059B801A994110D3104605
:105170001946224600F04AFB361A8F410197224613
:1051800001200021009F00F041FB38184D410090A4
:105190002046641E0028DFDC019B00982946324629
:1051A00007B0F0BD03460B439B0703D009E008C9D5
:1051B000121F08C0042AFAD203E00B780370401CC7
:1051C000491C521EF9D27047D2B201E00270401C55
:1051D000491EFBD270470022F6E710B513460A4677
:1051E00004461946FFF7F0FF204610BD30B50446CF
:1051F0000020034600E05B1C934203D2E05CCD5CE0
:10520000401BF8D030BDF8B502464A40D40F4200EA
:105210004B0052085B089A4202D2024608461146E9
:105220004A0023D0C30D4A00DDB2120EAD1A202D64
:1052300035DA49020126490AF6058A19002C00D000
:10524000524220214F1B1146B9402A411018C20D6D
:105250009A4221D0002C17D0012D08DCDA05801AE3
:10526000D20F8019D207DBB200F00CFBF8BDDA05D3
:10527000801A012340001B06C01880185A4280186B
:10528000CA0F1043490007E04908C2071143DA0575
:10529000801A80194008801800F0ECFAF8BD61000F
:1052A0000122511A001BF7E70122D2075140AAE759
:1052B0000122D2075040A6E770B502464A40D50FFA
:1052C00040004A00ED0740085208002814D0002A88
:1052D00012D0C40DD30D41020120C0055202490A6B
:1052E000520AE41A091812187D34914201D3641C41
:1052F00000E04900002C01DA002070BD002391423B
:1053000001D3891A0343400849000028F7D1002936
:105310000AD0914202D10121C90705E0914201D290
:10532000012101E00121C943E005C018401900F046
:10533000A1FA70BDF0B507460846584087B0C00FC7
:10534000049048000E46590040084908BC1A88419C
:1053500005D2384631461E4617460B4602465800CF
:10536000400810434CD0300D039040055900400DCB
:10537000490D0590401A0290402872DA1803012165
:10538000000B09050843019004980092002805D0FD
:1053900001995242002088410092019002984021D8
:1053A0000A1A0199009800F031FA05460C466B463E
:1053B00007CB00F04CFAC0197141039A0E0D00237F
:1053C000D71756401A467A40164344D0049A002A0A
:1053D0002DD0029A012A039A15DC1205C01A9141B8
:1053E00001263605001C7141D20F059ED20700939D
:1053F000019202962A46234600F08AFA07B0F0BDD1
:1054000038463146FAE71605224A0F46B218C01A46
:10541000B74101210905001C4F4100187F41114689
:1054200018187941E20F10436D19644113E0E20747
:105430006D0815436408C2071443039A0126120538
:10544000C01A91413605001C7141CE074008304317
:105450004908C01851412A46234600F04CFACDE7CE
:10546000FFE7049801224000C117121A00238B4164
:1054700004983146C417381AA141EEE730B401242C
:10548000E407634030BC55E730B40124E4076140D1
:1054900030BC4FE70000E0FFF0B51FB488B00B99B7
:1054A0000998002448400999C00F4900490809910A
:1054B000C0070B990090490049080B910999089879
:1054C000A64608431CD00B990A98084318D009989F
:1054D00001244000420D4800410D099824050003B5
:1054E000000B204309900B980003000B20430B9006
:1054F00050181C494018002201901446104605E03F
:10550000002001460DB0F0BD032801DA034600E09B
:1055100003239C46C11A0AAE0AE05F0008ADED5BAA
:105520004F00F75B7D430027AA187C41491C5B1E96
:105530006145F2DD410004AB5A522104120C0A43CA
:10554000240C401C0828DFDB01980290009970466B
:1055500001910090059B049A0799069800F0D8F9EC
:10556000D0E700000DFCFFFFF0B50C465C4085B0B5
:10557000E40FE40703944C000026640859009446A5
:10558000490802460296224321D062460A431ED0B1
:105590006200570D4A000E032303550D01240246F5
:1055A0002C492405781B1B0B360B4018234326433C
:1055B000614600901C46501AB44103D30098401C29
:1055C000009002E0921800985B41002803DA002066
:1055D000014605B0F0BD00200121090507468646B9
:1055E00011E064461D46141BB54106D36546521BA7
:1055F000B341744607430C43A646CD07400849080B
:10560000284392185B4105460D43EAD110461843E2
:1056100013D06046194650407140084306D060469A
:10562000101AB34106D20122002306E00022012312
:10563000DB0702E00122D2435310009874460105B3
:10564000381C6141029C039D0019694100F053F927
:10565000BFE70000FD03000070B54B005B0803438B
:105660000BD04B005C0D002633466542B341D41786
:10567000AD1AA34102DB0020014670BD12053018AF
:10568000514170BDC217C10F504010B54018CA0734
:105690009623002100F0F6F810BD10B500229623E5
:1056A000114600F0EFF810BD0EB5C217C10F504003
:1056B000CA0740180021054B0293019200910A4647
:1056C0000B4600F025F903B000BD000033040000D4
:1056D0000EB505490291002100910A460B46019141
:1056E00000F016F903B000BD330400004100400291
:1056F0000122400AD205090E80187F2901DA002014
:105700007047962903DC9622511AC8407047963993
:105710008840704770B5CD0F4A0009030123090B7B
:105720001B0519430B4BED070024520D9A4201DA79
:10573000002070BD074B34339A4203DC9A1A00F004
:1057400075F802E00449511888402C43F1D04042DA
:1057500070BD0000FF030000CDFBFFFF4A000903FE
:105760000123090B1B051943094B10B5520D9A4231
:1057700001DA002010BD064B34339A4203DC9A1A3A
:1057800000F054F810BD03495118884010BD0000C6
:10579000FF030000CDFBFFFFC20FD207400040080F
:1057A0000BD0C10D0723DB01C91840020905400ACF
:1057B0001143C2084007114370470020014670475B
:1057C000CB0FDB07490010B5490802460A4307D052
:1057D0000A0D07240903E401090B121B002A01DC4E
:1057E000002010BDC900440F0C43C100E018D205D1
:1057F000801800F03FF810BD0122D207002800DB1E
:10580000101A002900DB511A8142704710B5202A76
:1058100004DB0146203A9140002010BD9140202336
:105820009C1A0346E3401943904010BD10B5202A4E
:1058300004DB0846203AD040002110BD0B46D3407F
:10584000D0402024A21A91400843194610BD10B53B
:10585000202A06DBCB170846203A1041C1170B431C
:1058600006E00B461341D0402024A21A9140084381
:10587000194610BD002904DA401C490001D1400836
:105880004000704770B40024050C05D110240004BA
:1058900002D1002921D01124050E01D100020834C3
:1058A000050F01D10001241D850F01D18000A41C2A
:1058B000002801DB4000641C002908D020252E1B95
:1058C0000D46F540A14000D00121294308430106BF
:1058D0001B1B000ADB1D02D5002070BC7047DB05D6
:1058E000181880180029F8DA401C4900F5D170BC5E
:1058F00040084000704710B5002B08DA0024401C17
:10590000614192185B411A4301D14008400010BD2B
:10591000F0B51FB482B005460C0003D0084604F071
:1059200069FA02E004F066FA20300246009021464F
:105930002846FFF76BFF049B059A04460F46184361
:105940001143084314D0184610431BD0009840213F
:105950000A1A18460599FFF769FF05460E46009A90
:1059600005990498FFF752FF084305D0012004E091
:105970002046394607B0F0BD0020C11705430E434D
:105980002C43374300990E986305401A7905E40AC1
:1059900000220C43FD0A0A3002D500200146E9E747
:1059A0000105101969410C9C0D9D00196941FFF713
:1059B000A2FFDFE710B5002904DB0124E407404221
:1059C0008C412146002B04DB1C460123DB0752429D
:1059D000A3418B4200D1824210BD000010B50029C6
:1059E00004DB0124E40740428C412146002B04DB08
:1059F0001C460123DB075242A341994200D1904249
:105A000010BD0000064C0125064E05E0E36807CCFA
:105A10002B430C3C98471034B442F7D3FFF754FBA8
:105A200068B5000888B5000870B58C180578401C6A
:105A30006B075B0F01D10378401C2A1106D1027855
:105A4000401C03E006780E70401C491C5B1EF9D117
:105A50002B0705D40023521E0DD40B70491CFAE706
:105A60000378401CCB1A921C03E01D780D70491C72
:105A70005B1C521EF9D5A142D8D3002070BD000096
:105A800038B50446064805490068FFF731FB604316
:105A900000E0401E00900028FBD138BD40420F00BE
:105AA0004C010020F8B50446006881688907890F19
:105AB000012902D10168C90722D18168114A102643
:105AC0001140012500290ED1816829438160012000
:105AD000FFF7D6FF00F0C8FF07460CE000F0C4FF58
:105AE000C01B0A2807D9606D30436065A06D28434C
:105AF000A0650120F8BD20680068C043C007EDD153
:105B00000020F8BD1700008010B5012005F024FB2F
:105B10000A4C1328A0700AD0E01C02F0FBFBE078CE
:105B2000A070332806D006490020C88710BD05F0B4
:105B30004BFB10BD02F0C0FB10BD000000000020B8
:105B4000840D002010B500231A4603E0845CE3189E
:105B50009BB2521C8A42F9D3D84380B210BD0000D8
:105B600010B5034800F036FD024800F033FD10BDCB
:105B7000A41600205C16002030B5446C1C252C4077
:105B80000125A540046C6560046863608368102B80
:105B9000036803D099600068C26030BD9A600068F5
:105BA000C16030BD10490120487202205E31487248
:105BB00003203C39487204200E3948720A4B0B49C5
:105BC0005A1C0878587149789971233318715971A2
:105BD000203318775977107551751A461E32107593
:105BE00051751076517670478411002034010020E1
:105BF00010B503F00BFB202003F0A6FB012004F0FE
:105C00001DFD002003F0A0FB044804F0BBFB04488A
:105C100004F082FE002004F0B7FE10BDF800002062
:105C20008380000070B505200121000700F010FFFF
:105C300000240D4D002800D02C6002210B4800F0FC
:105C400007FF002808D10A482C6000880A21484331
:105C50000849088004F022F8012000F031FE0220FB
:105C600000F02EFE70BD0000440100200004005032
:105C70001E010020300100207047000010B50849C7
:105C800000224A6107494B684C1523434B604B681F
:105C9000082423434B60C009C001026010BD00000E
:105CA000EC160020002002407FB500250C46064679
:105CB000039500F0D5FDE009029003A90196009537
:105CC000684600F065FD002804D000F09DFD00202E
:105CD00004B070BD00F098FD0120F9E710B5002375
:105CE00002E0C45CCC545B1C9342FAD310BD0000AC
:105CF00010B5214A00219069C305204804D54169A7
:105D0000022319434161911593699B0505D54369A8
:105D10000124234343616302194393695B0505D55D
:105D20004369082423434361E301194393691B0535
:105D300005D54369042423434361630219439369EE
:105D40009B0405D54369102423434361630219432F
:105D500093699B0304D5446920231C434461194380
:105D60009369DB0305D54369402423434361A002C3
:105D70000143916110BD000000200240EC1600209C
:105D800070B5054600F070FE0646184C0AE0681C27
:105D900008D0002D04D000F067FE801BA84201D976
:105DA000032070BDA069C007F1D1A069800701D5AB
:105DB0000220A061A069C00511D4A06980050ED49D
:105DC000A06940050BD4A069000508D4A06980042F
:105DD00005D4A069800302D4A069C00303D5FFF7EE
:105DE00087FF012070BD002070BD00000020024030
:105DF000F8B51746002605460C4600F031FD09E0CF
:105E000029460220226800F00DFD002804D1241D3F
:105E10002D1D361DBE42F3D300F0F6FCBE4201D26A
:105E20000020F8BD0120F8BD10B508490246002049
:105E3000054B497905E044001C5B944203D0401CAB
:105E4000C0B28842F7D310BDC61200206000002007
:105E500010B5094800F0C6FF80B2FFF739FC074AC9
:105E6000074BFFF719FB0022064BFFF77DFBFFF7FF
:105E700075FC80B210BD000018150020F853E3A592
:105E80009B843E4000408F40F8B5414CE0790028AB
:105E900001D0002000E00120E0713D493D48CA7971
:105EA0000275097A41753C490A780276497841764B
:105EB0003A48017837481330017005214172962025
:105EC00004F01AFD4B20C00004F030FD31490022DF
:105ED00013310C2004F0FAFD00210C2004F008FE20
:105EE000022004F059FD2E4D00210F2004F060FC2B
:105EF0002842A063F8D0A06B411C3BD0294E2A4F0A
:105F0000400439D58122D20100210F2004F0B3FDD5
:105F10000021102004F04CFC41061E48490E0022CE
:105F2000633004F099FC1B4D6335687A052820D155
:105F300002221949681DFFF759F9002819D1A87ADA
:105F4000607113480422691C4C30FFF72BF9E06C98
:105F500000F02EF8A0836079294642000B310846F4
:105F60007330FFF71FF9A08B318848433880022037
:105F70002070F8BD02F08EFC0C480188A08B05460D
:105F8000FFF7B6F83088414339806D1EA583F8BD10
:105F900060000020E5110020340100200E010020E7
:105FA00000D0272418010020160100201A0100202B
:105FB00010B504460E4800F015FF0E49C006C00E8D
:105FC000098805E02246C240D2070FD0401CC0B26B
:105FD0008842F7D3012005E02246C240D20705D00F
:105FE000401CC0B28842F7D3491EC8B210BD0000A1
:105FF000181500201A01002010B5084800F096FA84
:106000000A21064800F032FA044800F01DF9800524
:1060100003D5024800F01AF980B210BDBC1400206C
:10602000F8B52F4D00220121284600F016FDFFF79C
:10603000E3FFFFF732FB2B4E3146FFF73DF92A4CC9
:106040000122A0601146284600F007FD2749A068FC
:10605000002588423EDB2078254F002815D025708A
:10606000FFF7CAFFFFF719FB3146FFF725F9A060DC
:10607000FFF792FB00223B46FFF700FA00221D4B80
:10608000FFF70AFAFFF79CFB6060A068FFF784FB4C
:1060900000223B46FFF7F2F9174A184BFFF7FCF9CD
:1060A00006460F466068FFF777FB134A144B5242CF
:1060B000FFF7F2F932463B46FFF73CF9FFF780FB6A
:1060C00010496060884201DD616004E0FF21C9057C
:1060D000C84200D365606068FFF708FBC0B2F8BD36
:1060E0000004005000401B443C00002000006040C1
:1060F00000000C4000E064403333333333B33040AE
:10610000CCCCEC3F0000C842F8B50546044640350B
:10611000287C0026012808D0012028742068816886
:106120008907890F01290ED101E00220F8BD01681D
:10613000C90708D0606D2021084360650126002052
:1061400028743046F8BD616DFF220132914302226E
:1061500011436165C1688907890F0091C168890889
:106160008900C1602068816892071143816000F056
:106170007BFC07460EE000F077FCC01B0A2809D91B
:10618000606D022188431021084360650020287457
:106190000120F8BD206880680028ECDB2068C16819
:1061A000009A1143C160606D80088000401C6065EA
:1061B000C5E70000F8B506460D464036317C01299A
:1061C0000DD00121317401688A68520709D5416DEB
:1061D000202211434165002030740120F8BD0220C7
:1061E000F8BD174B6A68D80547109A42154C8A6A61
:1061F0002B6812D05B035B0B1A438A622968490340
:1062000005D5A1680143A1600A20FFF739FC286881
:10621000800312D5A06838430EE05B035B0B9A4302
:106220008A622968490302D5A1688143A160286870
:10623000800302D5A068B843A06000203074F8BD88
:106240000110000000270140406D70470068006C9D
:106250007047000070B5040006D0606D264600252A
:106260004036002802D006E0012070BDA5653574D7
:10627000204600F0D3F8606DC00603D4216888681A
:10628000400705D5606D1021084360653574EBE764
:10629000606DFF22013290430222104360658868DE
:1062A0008207920F5B48012A02D10A68D2072BD1DC
:1062B000032362689B079A4205D05B429A4202D050
:1062C0005B009A4209D10A69920092080A6121682A
:1062D0000A6963681A430A610CE00A69920092082D
:1062E0000A6181680F22920491438160816862682B
:1062F000114381602168CA6818239A43CA602168E3
:10630000CA68A3681A43CA60816801225206914391
:1063100081608168A28E5206114381602068816885
:10632000C90004D4816801221207114381602068EA
:10633000C168394A1140C1602069E168022825D04E
:1063400000200143204620300278037B52035B008B
:106350001A431143226B1143A26992031143E2696C
:10636000D20311432268D3681943D160616A0A4697
:10637000FF3AC23A05D0A26A11432268D368194392
:10638000D16042780121012A02D00BE00420D8E735
:106390000078002823D0606D202210436065A06D36
:1063A0000843A065E06B012820681FD00169C90778
:1063B00003D0016949084900016120684169C908A1
:1063C000C900416120684169A26B11434161A56523
:1063D000606D80088000401C6065002070BD2068F2
:1063E000C26801231B041A43C260DBE70269FF2372
:1063F0009B009A43026120680269236CA66C1A43D1
:10640000636C33431A430261206802690A430261E4
:10641000D3E70000002701401902FEFF10B586B047
:10642000044614216846FEF7D6FE0E4920688842CD
:1064300016D10D48416B421511434163C16A0122D7
:106440001143C162C06A6946104005900220009065
:1064500003200190002002900520000700F03CFA84
:1064600006B010BD0024014000100240F8B50446FB
:106470004069254640350E4608280BD02068C06884
:10648000C00709D0606D2021084360650020287492
:106490000120F8BD082700E00C2700F0E5FA009085
:1064A00011E0701C0FD0002E05D000F0DDFA00992D
:1064B000401AB04207D9606D04210843606500208E
:1064C00028740320F8BD206800683842E9D0606D68
:1064D00001214902084360652068C16809058A0FE7
:1064E0000C21002A1BD12022125D002A17D102683C
:1064F000120714D5826853070122002B08DB43687A
:106500008B434360606D130298431043606506E05F
:10651000606D202318436065A06D1043A065A069DD
:10652000002801D1206801600020F8BD70B5044644
:10653000216800208968490721D425464035297CF7
:1065400001291CD001212974E169012904D02046C8
:10655000FFF7A8FA002811D1616D0A4A1140FF2205
:106560000132114361650021A165297422681C2153
:10657000116021688A6804231A438A6070BD022072
:1065800070BD0000FEF1FFFF70B500240146203110
:106590004A79022A03D00421C163012418E0026869
:1065A00013680E25AB431360026813685B085B0039
:1065B0001360436C1C221340012215469D40036C5E
:1065C0005D604A7100220A71816B002900D0884702
:1065D000204670BDF0B4016C0D6801680C68466C13
:1065E0001C2304221E401746B7402F420ED06707D7
:1065F0000CD50C68A40602D40C6894430C60416C62
:1066000019408A40016C4A60016B1AE00227B740CA
:1066100002462F402032002F17D0A70715D50C684F
:10662000A40605D40C680A25AC430C600121517105
:10663000446C02211C40036CA1405960002111717F
:10664000C16A002918D0F0BC08470827B7402F427C
:1066500012D0240710D50C680E25AC430C60446C96
:1066600001211C400B46A340046C6360C16351715F
:1066700000211171416BE4E7F0BC704770B5040074
:106680003CD01F48256814212818FEF731FD8000F2
:1066900060641C482064022120462030024641717B
:1066A00029681948E3680140A068666918432369AE
:1066B00033431843A3691843E3691843236A184313
:1066C000084328600121A0688903884210D00D4842
:1066D0008030836A656C1C210D400F26AE40B343A9
:1066E0008362656C63680D40816AAB400B438362D3
:1066F0000020E06301215171107170BD012070BD57
:10670000F8FFFDBF000002400F80FFFFF8B5044610
:106710008C46203001790025012909D00126067117
:1067200041790027012905D0077102252846F8BDC7
:106730000220F8BD02214171E76320680168490821
:106740004900016061462046FFF716FA206B0028D9
:106750002068016801D00E2205E004229143016007
:10676000206801680A2211430160206801683143F2
:106770000160DBE770B5044600F076F90546601C61
:1067800000D0641C00F070F9401BA042FAD370BD29
:10679000F8B51A4E0546307C0F46012807D0012077
:1067A00030741748FFF7ECFA010002D021E0022014
:1067B000F8BD0020C04338606C6814E02046FFF745
:1067C0005DFA0F48FFF7DCFA01460E4842680823DD
:1067D0009A434260426843159A434260002901D0BF
:1067E0003C6006E08034A8686A68C0018018A04256
:1067F000E4D8002030740846F8BD0000EC160020F4
:1068000050C30000002002400548416802221143A5
:10681000416041680122114341600020704700003F
:1068200000200240F8B50C4C1646207C0F4601288B
:1068300008D0012020740948FFF7A2FA002500289B
:1068400002D006E00220F8BD65613E600348FFF714
:1068500097FA2574F8BD0000EC16002050C3000024
:1068600011484168C9070BD0EFF3108172B60F4A87
:10687000C2600F4AC26081F310884168C9070ED117
:10688000416889070DD5EFF3108172B6094A02619C
:10689000094A026181F310884068800701D5012010
:1068A000704700207047000000200240EFCDAB8908
:1068B00005040302BFAE9D8C16151413704700002B
:1068C00010B504494A69024202D04861FFF7F6FF59
:1068D00010BD000000040140F8B500230124A2E02F
:1068E00027469F403A4070D04D68022D01D0122DAE
:1068F00014D1DD08AD002D1800952D6A5E07AC4659
:10690000F50E0F26AE46AE406546B543AC460E6961
:106910007546AE4065462E43009D2E624D68012DA2
:1069200005D0022D03D0112D01D0122D16D185686E
:106930000326AC465D00AE46AE406546B543AC4668
:10694000CE687546AE4065462E43866046680D7932
:10695000BE43ED06ED0F9D403543456006685F0080
:106960000325BD40AE46AE430D79B446AE07B60F23
:10697000BE4065462E430660C6687546AE438D68C8
:10698000BD403543C5604D68ED004BD5294D6E6B5C
:1069900026436E639E08284DB6007519AC46AD6857
:1069A0009E07360F0F27B740BD4305273F07B84264
:1069B00001D1002715E0214FB84201D1012710E095
:1069C0001F4FB84202D102270BE02BE01D4FB84207
:1069D00001D1032705E01C4FB84201D1052700E093
:1069E0000627B7402F436546AF60184D2E684F68A5
:1069F0009643FF0300D516432E606E684F6896439A
:106A0000BF0300D516436E60AE684F689643FF0221
:106A100000D51643AE60EE684F689643BF0200D5BE
:106A20001643EE605B1C0A681546DD4000D057E750
:106A3000F8BD0000001002400000014000040050BA
:106A400000080050000C0050001C005000040140E1
:106A50000069084000D001207047002A01D0816100
:106A6000704781627047000001480068704700006D
:106A70004801002002480168491C0160704700007D
:106A80004801002010B50848002401684022114345
:106A90000160204600F00AF8002801D0012401E03E
:106AA00000F0CCF9204610BD0020024070B505462C
:106AB00009487D210024C9000068FEF719FB00F099
:106AC00061FE002801D0012404E000222946501E66
:106AD00000F0D4F9204670BD4C010020704770478B
:106AE000F8B53A4C01266078401C6070E670208C46
:106AF000401C2084608902F0F1FB354FF888FEF7D6
:106B0000CCFD3449FEF7D8FB334D00902968FEF7E1
:106B10007AFB2860E16AF005814203DB0098FEF70A
:106B2000C7FBE06202212D48FFF792FF002808D042
:106B3000002020632A492F682A488F4227DD0670EB
:106B400027E0F888FEF7A9FD2249FEF7B5FB216B87
:106B5000FEF759FB244920638842EBDBE0790028EB
:106B600013D000211A484030818004F045FC0121F7
:106B7000002289021948FFF770FF7D200001FFF70E
:106B8000F9FD1B491948C860D4E70121EAE7002153
:106B90000170207A401EFEF775FD3946FEF72CFE87
:106BA00006D82079002803D01248C1793143C17139
:106BB000207AFEF772FD2968FEF71EFE04D22079C6
:106BC000002801D004F08CFAF8BD00000C01002070
:106BD000840D002000007A4444010020000400508D
:106BE00000004040660000200000A0400400FA05BC
:106BF00000ED00E0F8110020704770B505000DD0E1
:106C000002202C462034A073284601F01FFC2846A1
:106C100000F0BEF80020A073607370BD012070BD4D
:106C20007047704710B5044600680168C943C9073A
:106C300008D18168C943C90704D1012141602046B8
:106C4000FFF74EFF20680168C943890708D48168AF
:106C5000C943890704D4022141602046FFF73EFF63
:106C600020680168C943490708D48168C9434907B6
:106C700004D404214160204600F0DEF82068016859
:106C8000C943090708D48168C943090704D4082106
:106C900041602046FFF7B0FF20680168C943C9067C
:106CA00008D48168C943C90604D410214160204634
:106CB000FFF715FF20680168C943890608D4816879
:106CC000C943890604D4202141602046FFF7A9FF6B
:106CD00020680168C943490608D48168C943490648
:106CE00004D4402141602046FFF79AFF10BD000008
:106CF000F8B5040005D025462035A87B002802D031
:106D000006E00120F8BD00206873204600F052F82C
:106D10000220A8732068C26884466368012B04D0EF
:106D20000120A16AC005814201D11E20824315487D
:106D30006169814201D0144802401448A6680240AB
:106D400018463043676A266A3E433043A66A30439A
:106D50001043012B03D00122D205964203D12369AF
:106D6000E2681A431043074A914205D0A2691143D1
:106D7000E2690243084610436146C8600120A873D7
:106D80000020F8BDFFFF00003F1FFFFFF8F119FFD3
:106D900010B500680549884207D10548816B490054
:106DA000490881630D2000F055F810BD007C0040BB
:106DB0000010024010B50068084988420CD108480C
:106DC000816BC20411438163002201210D2000F078
:106DD00055F80D2000F048F810BD0000007C004080
:106DE000001002400068C0697047000070B50224BE
:106DF000034620339C730F4C2568E6043543256019
:106E00000468E568B6123543E5600568AE6801249C
:106E10002643AE6005682E6926432E610568A96188
:106E200001684A61006801690422114301619C7391
:106E3000002070BD00040140704700000448416B11
:106E4000012211434163816B020411438163704746
:106E500000100240C106C90E0120884001490860A7
:106E60007047000080E100E0C106C90E01208840A3
:106E7000014908607047000000E100E010B501F032
:106E8000E7FC10BD02494A6882434A60704700002F
:106E9000007000400248016882151143016070478C
:106EA0000070004002494A6802434A60704700008F
:106EB0000070004005480168022211430160044847
:106EC000016904221143016130BF70470070004026
:106ED00000ED00E00A4B1A689208920002431A6023
:106EE00008480369042213430361012906D040BF07
:106EF00020BF20BF016991430161704730BFF9E7AE
:106F00000070004000ED00E0F8B504460078544DF4
:106F1000800672D5524E0027403EB06BC00004D4AC
:106F2000B06BA9050843B06301274E480168C90545
:106F300011D40168821511430160FFF795FD00909F
:106F400005E0FFF791FD0099401A642837D84548BD
:106F50000068C005F5D532680321090560680A405C
:106F60000140914208D08103890F032904D131687F
:106F7000890301D50120F8BD2A69032109040A40CB
:106F800022D0084090421FD0207880061CD5286966
:106F90002A6988430121C9040A432A612A698A436C
:106FA0002A612861C0050FD5FFF75EFD009008E05B
:106FB000FFF75AFD0099411A2B48814201D903205D
:106FC000F8BD28698005F3D561688803800F032820
:106FD00005D132680005824301400A4332602869C6
:106FE000032261681204114008432861002F04D075
:106FF000B16B012000078143B1632078C00705D041
:10700000E868A168800880000843E860207880076D
:1070100005D5E8680C218843E1680843E8602078DA
:10702000400706D5E868032189028843216908439F
:10703000E8602078000706D5E86803210903884343
:1070400061690843E8602078000606D5E8680321F6
:1070500089048843A1690843E8600020F8BD000066
:10706000401002400070004088130000F8B50E4642
:1070700005007DD053480068C007C00FB0420AD257
:107080005048016849084900314301600068C00761
:10709000C00FB04271D128784B4C800705D5E0680D
:1070A000F0218843A9680843E0602878C00752D0DF
:1070B0006868022817D0032818D02168012818D042
:1070C0008905002959DAE168890889000143E160EE
:1070D000FFF7CAFC69680746022912D003291CD0B1
:1070E000012926D033E021688903EAE72168890174
:1070F000E7E74907E5E7FFF7B7FCC11B33488142E3
:1071000023D8E0680007800F0228F4D123E0FFF7BE
:10711000ABFCC11B2D48814217D8E0680007800FE7
:107120000328F4D117E0FFF79FFCC11B27488142D9
:107130000BD8E0680007800F0128F4D10BE0FFF7BF
:1071400093FCC11B2148814201D90320F8BDE068AE
:107150000007800FF3D11B480168C907C90FB1426E
:107160000DD901684908490031430160006800E019
:1071700003E0C007C00FB04201D00120F8BD28785D
:10718000400706D5E068072109028843E9680843FB
:10719000E0602878000707D5E0680721C902884326
:1071A0002969C9000843E06000F036F8E168084A40
:1071B0000906090F515CC840064908600020FFF726
:1071C00075FCF8BD0020024000100240881300004A
:1071D00002B500084C010020044805490068C96850
:1071E000044A4905490F515CC84070474C010020D2
:1071F000001002401BB50008044805490068C96832
:10720000044A8904490F515CC84070474C01002072
:10721000001002401BB5000810B5184AD1680C20B8
:10722000084004280BD0082810D00C2810D0506833
:107230000004410F0120C003491C884010BD1068A4
:10724000C00601D50E4810BD0E4810BD0E4810BD39
:1072500088020E4B000F185C0902D368890F491C85
:10726000DB0301D5084A05E01268D20601D5044ABD
:1072700000E0044A5043FDF73BFF10BD0010024000
:1072800000093D000024F40000127A0012B5000845
:10729000FEB505007ED0FE4CE7680C20E66807408E
:1072A0000120000406402878C00747D0082F05D0E9
:1072B0000C2F0AD101200004864206D120688003E9
:1072C0003CD568680028E5D038E0012069680004F2
:1072D000814203D121680143216011E0052301228D
:1072E0001B0492049942216802D111432160F1E705
:1072F0008143216021680140009120689043206013
:10730000686800280DD0FFF7AFFB009005E0FFF79D
:10731000ABFB0099401A64287AD820688003F6D520
:107320000CE0FFF7A1FB009005E0FFF79DFB009943
:10733000401A6428F0D820688003F6D428788007A3
:1073400055D50923E868042F0DD00C2F01D1002E4C
:1073500009D000283BD02168994301432160FFF701
:1073600083FB064627E02168490701D5002891D014
:1073700061681F22120291432A691202114361605F
:107380002168994301432160FFF746FFE168090640
:107390000A0F00E079E1BF49895CC840BE49086036
:1073A0000020FFF783FB002872D120E0FFF75CFB91
:1073B000801B0228B0D820684007F7D560681F21DD
:1073C0000902884329690902084360600FE02068C8
:1073D000400840002060FFF747FB064604E0FFF747
:1073E00043FB801B022897D820684007F7D42878F1
:1073F000C0065FD5002F0CD0A869002849D02068AE
:10740000FF21013108432060FFF72EFB06462DE0E7
:10741000C0E02068800502D5A8690028A7D0606870
:10742000072149038843296A084360606068297F0F
:107430000002000A090608436060286A410B012027
:10744000C003491C8840E16809060A0F9149895C1C
:10745000C840914908600020FFF728FB002817D199
:1074600028E0FFF701FB801B0228A3D820688005D5
:10747000F7D56068072149038843296A084360609B
:107480006068297F0002000A09060843606011E075
:10749000E1E02168FF20013081432160FFF7E4FA39
:1074A000064604E0FFF7E0FA801B022872D8206845
:1074B0008005F7D42878794E000724D5686900281C
:1074C000306910D0012108433061FFF7CDFA0090F8
:1074D00005E0FFF7C9FA0099401A02285AD8306926
:1074E0008007F6D50FE0400840003061FFF7BCFA96
:1074F000009005E0FFF7B8FA0099401A022849D831
:1075000030698007F6D42878400765D500200290BE
:10751000A06BC00006D4A06B012109070843A0633B
:10752000012002905E480168C90511D401688215E6
:1075300011430160FFF798FA009005E0FFF794FA15
:107540000099401A642825D855480068C005F5D52B
:10755000FF20AA680130824203D1316901433161C1
:1075600011E001218902002A07D005231B029A425B
:1075700003D132690A433261EFE7326982433261F3
:10758000306988433061A86800280FD0FFF76CFA93
:10759000009007E05EE0FFF767FA0099411A414862
:1075A000814257D830698005F5D50DE0FFF75CFAC8
:1075B000009006E0FFF758FA0099411A39488142D5
:1075C00048D830698005F5D40298002804D0A06B13
:1075D000012109078843A063686A002864D00C2F42
:1075E0003ED0012636060228206805D0B043206030
:1075F000FFF73AFA05462FE0B0432060FFF734FA70
:10760000074604E0FFF730FAC01B022822D82068A2
:107610008001F7D4E96AA86AE2680843296BFD2370
:107620001B049A4311430843E06020683043206004
:10763000FFF71AFA054604E0FFF716FA401B022886
:1076400008D820688001F7D52EE0FFF70DFA401B1F
:10765000022801D90320FEBD20688001F5D423E073
:107660000128F8D0E06801210904AA6A014091428A
:107670000BD10F218904EA6A0140914205D103210F
:1076800089050840296B88420ED00120FEBD00000C
:107690000010024002B500084C01002040100240DA
:1076A00000700040881300000020EFE770B5040070
:1076B00007D0002625464035A662687C002802D007
:1076C00005E0012070BD2E74204600F02FF8022046
:1076D000687420680168402291430160A168606875
:1076E00022690843E16811430843616901220843A4
:1076F000A169520211400843E1690843216A084325
:10770000A16A084321680860A0690421000C0840B0
:10771000616A0843216848602068C169920091430A
:10772000C161666501206874002070BD10B586B027
:10773000044614216846FDF74EFD10492068884232
:1077400019D10F48416B821411434163C16A012270
:107750001143C162C06A002110400590E0200090F2
:1077600002200190032003900291049105206946B4
:107770000007FFF7B1F806B010BD0000003001406F
:1077800000100240094910B5401E884201D901206D
:1077900010BD074C60610321081F01F059F800205B
:1077A000A06107202061002010BD0000FFFFFF0046
:1077B00000E000E0F0B502462032137E012B15D028
:1077C000012717760223537605686C68AB6870262C
:1077D000B4430E68496826438024A34319436E606E
:1077E00000688160577600201076F0BD0220F0BD61
:1077F00070B5040005D025462035687E002802D0EB
:1078000006E0012070BD00202876204600F00AF82E
:1078100002206876211D206801F01AFE012068769A
:10782000002070BD006801218907884204D1034807
:10783000816B0122114381637047000000100240F8
:10784000F8B5054604462035287E012817D00126C4
:107850002E7602206876226890687727FF23B84347
:107860001B02984390600A68502A31D00EDC202A0F
:107870004BD006DC002A48D0102A3AD145E002203D
:10788000F8BD302A41D0402A33D136E0602A27D0D3
:10789000702A12D001200003121A2AD0824228D165
:1078A000CB684A688968206801F00BFE206881680F
:1078B00001229203114381601BE0CB684A6889680A
:1078C000206801F0FEFD216888683843886010E078
:1078D000CA684968206801F06EFE5021206806E001
:1078E000CA684968206801F077FE6021206801F0CD
:1078F000F3FD6E7600202876F8BDCA6849682068D6
:1079000001F059FE40212068F1E711462068EEE7BA
:1079100010B586B0044614216846FDF75CFC0121D1
:1079200020688907884212D10A49CA6A02200243A4
:10793000CA62C96A0190014005914102009100218B
:1079400002910391049069460348FEF7C5FF06B013
:1079500010BD00000010024000040050F8B50646BB
:1079600004462036307E0D4601280DD001203076A9
:10797000022070760427002A08D0042A16D0082A8C
:107980002AD00C2A4DD137E00220F8BD206801F042
:10799000ABFD2068816908221143816120688169FB
:1079A000B943816120688169EA6812E0206801F0CA
:1079B000B3FD206882690121C9020A4382612068FF
:1079C0008169012292029143816120688169EA689C
:1079D00012021143816124E0206801F0B6FD2068A5
:1079E000C26908210A43C2612068C169B943C16103
:1079F0002068C169EA6812E0206801F0C1FD2068D2
:107A0000C1690122D2021143C1612068C26901210A
:107A100089028A43C2612068C169EA68120211437F
:107A2000C1610120707600203076F8BD70B5040089
:107A300005D025462035687E002802D006E00120CA
:107A400070BD00202876204600F00AF802206876F3
:107A5000211D206801F0FCFC01206876002070BD2B
:107A6000704710B504460068012201F01DFD206832
:107A700081684907490F062903D001680122114393
:107A80000160002010BD000010B50446006800220F
:107A900001F00AFD2068016A054A114203D101681C
:107AA000490849000160012020346076002010BDA3
:107AB0001111000070477047F8B502680446D0699C
:107AC0001168936805072D0F5BD0DD07ED0FFF26CA
:107AD00021360E402E4367D0C60706D0CE0504D50A
:107AE00001261662E26F3243E2678707022204260C
:107AF000002F06DADF0704D027683A62E76F3743C2
:107B0000E767470706D5DB0704D023681E62E36FEB
:107B10001343E367020709D520220A402A4305D010
:107B2000236808221A62E36F1343E367E26F002AB7
:107B30002FD0800606D5880604D5216E002901D0F5
:107B400020468847E06F21688968490601D400070C
:107B500024D5204601F0E6FE20688168490619D543
:107B60008168402291438160E06E002812D0204954
:107B70008163E06EFEF708FD00280AD0E06E816B9D
:107B800006E0850610D58D060ED5216E1CE0204638
:107B90008847F8BD2046FFF78EFFF8BD2046FFF767
:107BA0008AFF0020E067F8BDC50208D55B0206D554
:107BB0000120000510622046FFF77CFFF8BD030698
:107BC00005D50B0603D5616E0029E0D1F8BD40064E
:107BD000FCD54806FAD51368204640218B43136034
:107BE000202161670021616600F069F9F8BD00009D
:107BF0008198000810B5040003D0606F002802D0FF
:107C000007E0012010BD002170200155204600F042
:107C100027F824206067206801684908490001604E
:107C2000204601F0C9FE0128ECD0606A002802D08D
:107C3000204601F007FD206841680922D2029143E5
:107C40004160206881682A22914381602068016830
:107C5000012211430160204601F05AFD10BD0000D1
:107C6000F0B587B0064614216846FDF7B4FA2C49F2
:107C70003068884251D12B48416B01229203114355
:107C80004163C16A01221143C162C06A00251040EC
:107C900005900320400200900220032701A9A1C102
:107CA00004200490052069460007FEF715FE1F4CCE
:107CB0001D48A560E56081C48027E560A76020209D
:107CC000256160610002A0611848083CFEF7D6FCFF
:107CD000002801D0FDF7D0FFF466A662144C1248CC
:107CE0002146143820600320606010200831A1C1B3
:107CF0006561A561E56120462562FEF7BFFC0028AD
:107D000001D0FDF7B9FFB466002201211B20A66255
:107D1000FFF7B4F81B20FFF7A7F807B0F0BD00008D
:107D20000038014000100240300002405C16002084
:107D3000A4160020F8B50446806F20284DD10029F4
:107D40000BD0002A09D00123A0681B03984206D15A
:107D50002069002803D1C80701D00120F8BD2546BD
:107D60006035287C012838D00120287458206165AE
:107D700002530026E6672220A067E06E002819D093
:107D80001749C162E16E17480863E16E16484863FF
:107D9000E06E13468663676D21683A462431E06ED3
:107DA000FEF7B4FC002805D01020E0672E742020D8
:107DB0006067D2E72E7420680168FF220132114308
:107DC0000160206881680122114381602068816818
:107DD0004022114381600020F8BD0220F8BD000060
:107DE000DD9800081B9900089598000870477047B7
:107DF000FFB50446406F83B017460D4620285CD17E
:107E0000002D0AD0002F08D0A168C001814207D1FF
:107E10002069002804D1E80702D0012007B0F0BD96
:107E2000204660300290007C012846D00298012153
:107E300001740020E06721206067FEF715FE2646EA
:107E400040360190378277820120A1680003814289
:107E500002D12069002802D02F46002511E000271A
:107E60000FE000228021204601F0BAFE002815D143
:107E7000002F15D02168387888627F1C708A401ED8
:107E80007082708A019B002806980090E9D1002238
:107E90004021204601F0A4FE002808D00320BDE7C1
:107EA00028882168C005C00D8862AD1CE6E7202047
:107EB0006067029900200874B0E70220AEE77047BF
:107EC00001490248C160FDE70400FA0500ED00E049
:107ED00070B586B014216846FDF77DF90F4801247E
:107EE000818B002900D18483808B012805D0022852
:107EF00001D100F035FC06B070BD0122084E95029C
:107F000029463046FEF7A9FD002102910391009514
:107F1000019469463046FEF7DFFCECE70C010020D7
:107F20000004005010B50524240700220421204637
:107F3000FEF793FD002208212046FEF78EFD0A2061
:107F400002F0D9F9012204212046FEF786FD0A201D
:107F500002F0D1F9002204212046FEF77EFD10BD7B
:107F600010B505242407002204212046FEF775FDE4
:107F7000012208212046FEF770FD0A2002F0BBF91D
:107F8000012204212046FEF768FD0A2002F0B3F921
:107F9000002204212046FEF760FD10BDF8B5002444
:107FA0000526074625463607002204213046FEF7FF
:107FB00054FD0A2002F09FF9012204213046FEF709
:107FC0004CFD6006040E08213046FEF741FD0028F6
:107FD00001D0641CE4B2052002F08DF96D1CEDB2F5
:107FE000082DE1D3002F03D0FFF79CFF2046F8BDFA
:107FF000FFF7B6FFFAE770B50526054636070022FB
:1080000004213046FEF729FD0024E80901D00122B1
:1080100000E0002208213046FEF71FFD6806050E2D
:108020000A2002F068F9012204213046FEF715FD0E
:108030000A2002F060F9002204213046FEF70DFD0F
:108040000A2002F058F9641CE4B2082CDDD370BD9C
:1080500010B505242407012208212046FEF7FDFC67
:10806000012204212046FEF7F8FC002208212046C8
:10807000FEF7F3FC0A2002F03EF90022042120461C
:10808000FEF7EBFC10BD10B50524240700220421E7
:108090002046FEF7E2FC002208212046FEF7DDFC28
:1080A0000A2002F028F9012204212046FEF7D5FC1F
:1080B000012208212046FEF7D0FC0A2002F01BF91D
:1080C00010BD70B505252D07002401220821284682
:1080D000FEF7C3FC062002F00EF901220421284617
:1080E000FEF7BBFC062002F006F907E0641CE4B2D0
:1080F000FA2C03D9FFF7C7FF012070BD08212846DD
:10810000FEF7A6FC0028F1D1002204212846FEF744
:10811000A4FC002070BD0000F8B501F029FB01F0BF
:1081200063FB56480068C069554E564F800700D51E
:10813000FE60FDF78DFE5449544D898F544C002943
:1081400029D054490A7801218902002A05D0012A40
:108150000ED0022A10D0032A1DD1A08B01282DD0C9
:10816000022818D1454808213C38FFF78DFC12E061
:10817000FF22F5329042F0D2A08B01281CD00228B9
:1081800004D008E02846FEF768FC04E03B480821DC
:108190003C38FFF766FC0121C9023C48FEF758FC59
:1081A000002500282CD03C480560FDF739FF2070E1
:1081B000A079002804D007E00022E3E70122E1E7EC
:1081C0000120A07101F06AFD2078632806D9002201
:1081D00008212E48FEF741FC012205E0012208217A
:1081E0002A48FEF73AFC002201210520C9030007B6
:1081F000FEF733FC244C4034A08C012803D01CE053
:10820000A5710022EBE725486946088072B68021F7
:108210002348FDF749FD002804D002226946204882
:10822000FDF7E6FD62B61FA001F0D4FDA58403F0C2
:10823000E3F8642002F058F8FE60608C012808D151
:1082400011486584058003F0D7F8642002F04CF8EB
:10825000FE60208C012806D1258403F0CDF864202F
:1082600002F042F8FE600848124A0188914202D1A9
:10827000C088002800D1FE60F8BD0000DC15002099
:108280000400FA0500ED00E0840D00200004005019
:108290000C0100207100002044010020AAAA000067
:1082A000384A0008BDF8C8EBC9FDBCB6C4A3CABDB6
:1082B0000D0A0000AA55000010B53721202000F05B
:1082C00070F80321212000F06CF84021222000F0FA
:1082D00068F80821232000F064F8AA21302000F07B
:1082E00060F80A4801210187322000F05AF8012184
:1082F000332000F056F85F21202000F052F80448A7
:1083000000F008F80A2001F0F6FF10BD840D0020EF
:108310000300002010B501460F2000F021F80028CE
:1083200000D0012010BD10B50446FFF791FE3220A9
:10833000FFF761FEFFF7C5FEE0B2FFF75CFEFFF757
:10834000C0FEFFF785FE3320FFF755FEFFF7B9FEAD
:108350000020FFF723FE0446FFF795FE204610BDE0
:1083600010B50C46FFF7DFFF2070012010BD70B57F
:108370000D460446FFF76CFE3220FFF73CFEFFF788
:10838000A0FEE0B2FFF737FEFFF79BFE2846FFF79F
:1083900032FEFFF796FEFFF776FE0A2001F0ABFFF4
:1083A00070BD10B5FFF7E3FF012010BDF8B5214CFB
:1083B00045882585C28862850389A3858189E185F1
:1083C000408920866D435243A8185B43C018494337
:1083D000FCF7A4FEFDF768F902F072FD0022164BCF
:1083E000FDF75AF8636E226EFDF748F8274680378E
:1083F00003C7E08D083F4043FDF756F905460E469A
:10840000208EFDF765F9E36DA26DFDF745F82A466C
:108410003346FDF7A9F802F053FD0022064BFDF7A5
:108420003BF8636E226EFDF729F8F960B860796950
:108430003869F8BD600000200000244010B50248F3
:10844000FEF7F0FB10BD000018150020FEB5044635
:10845000002572B60068394A831804D13849CD68BE
:10846000032189040D4081680191C168009141692F
:108470008669002B08D132484038836AC7043B43E1
:108480008362836ABB4383620846304348D02B48EB
:108490002368C34205D12A48C36803229204934348
:1084A000C360002917D02068026901231A430261C2
:1084B00020684161FEF7D8FA0746FEF7D5FA216831
:1084C000C01B0968090703D47D21C9008842F4D97B
:1084D000216808204860002E17D020680169012219
:1084E0001143016120688661FEF7BEFA7D270646CA
:1084F000FF00FEF7B9FA2168801B0968C90601D49C
:10850000B842F6D92168102048600C482168C14261
:1085100006D10B48C1680322920491432943C160EC
:108520002068016949084900016121680198886053
:1085300021680098C86062B6FEBD00000084FFBFDD
:10854000401002401CB5002116480091144A0191C8
:108550000260C163120542608160072282630122CA
:1085600002610246C16020321170FF235170C23394
:10857000436281621173016381610422416342613C
:10858000C161FDF767FE08480090801301906946BD
:108590000448FDF70FFE00210248FDF7B5FD1CBDA4
:1085A00000240140BC1400200200000408B5084863
:1085B000016B012211430163006B01211040009007
:1085C00000220A20FEF75AFC0A20FEF74DFC08BDE7
:1085D00000100240F0B587B014216846FCF7FBFD9F
:1085E0004748C26A04210A43C262C26A0A4005922D
:1085F000C16A80263143C162C16A31400591C16AB6
:1086000001242143C162C16A21400591C16A02254A
:108610002943C162C06A22462840059005201C21DA
:108620000007FEF71AFA012236493748FEF715FA15
:10863000002236493448FEF710FA91210520002225
:1086400009020007FEF709FA3148019000270520CA
:108650006946029700940007FEF73EF90C2000904F
:10866000112001900320039005200297694600071E
:10867000FEF732F910206A46039591C2052069463B
:108680000007FEF729F91120019002976946039728
:1086900000941D48FEF720F91E4801906946009598
:1086A00002941948FEF718F9E00200906946019714
:1086B00002951548FEF710F91748694691C16946B9
:1086C00011480397FEF708F991200002694691C10D
:1086D0000520694600070397FEF7FEF869460A4839
:1086E000019700960294FEF7F7F800220121052079
:1086F000FEF7C4FB0520FEF7B7FB07B0F0BD000096
:108700000010024001020000000400500830000088
:1087100000001110000021100832000010B50F4CAD
:108720000D482060FF20053060600020A060E06000
:1087300020616061E0610121206249026062A16103
:10874000A0620720E0622046FEF7B0FF20680168C3
:1087500040221143016010BD003001404815002047
:1087600010B58AB0002404940594069407940894E4
:1087700001211848099400940194029489070394F4
:108780000160092184604160046113494461C16052
:10879000FFF72EF801200003049004A90D48FFF70D
:1087A0004FF80C48FFF742F9089408A909480994C2
:1087B000FFF700F86020009008480190029408221A
:1087C000694603940348FFF7C9F80248FFF7A0F889
:1087D0000AB010BDA015002093040000570200004D
:1087E00000B585B014216846FCF7F5FC164815491C
:1087F0000160E1214902416000218160C1600161A5
:1088000081610C22C161426101623021416201211A
:10881000090381634900C163FFF7ECF9012080027D
:108820000090022001900120029003200390042078
:108830000490052069460007FEF74EF801F028FA7B
:1088400005B000BD00380140DC1500207047000075
:108850008307FF22DB0E9A408907090E9940002802
:108860000BDA0007000F0838830808489B00181827
:10887000C36993430B43C3617047830804489B005B
:108880001B181868904308431860704700ED00E01B
:1088900000E400E0BFF34F8F04490348C860BFF312
:1088A0004F8F00BFFDE700000400FA0500ED00E077
:1088B000F0B58DB0962002F01FF84B20C00002F0FA
:1088C00035F8FF4F00247C70B87B0C2801D30B20B7
:1088D000B8730122052051020007FEF7BEF8B87BED
:1088E00078737871F748BC70F74D00782870F748B6
:1088F000022100782871F648FEF7AAF8002865D012
:108900000020B979F04D49000843E871786BE870B0
:10891000401C786378792946A8724200CE31084617
:10892000C338FCF73FFC062068727879E94980007B
:1089300042190B78D372497811732A46133AE049E9
:1089400004928B7F1375C97F5175002229460F3021
:1089500002F0BCF87879002180000F3002F0C8F8EE
:10896000022002F019F8EC713C74BC7201203873DB
:10897000FC72D948FEF736FA78840546BC707879DF
:10898000FCF7A6FED54AD64BFCF786FD01F048FC65
:108990000022D44BFCF7CEFCFCF7E0FE0006C10C35
:1089A000481980B20121C903B884884201D3401A12
:1089B000B884CD483864F878401CF870C648FEF793
:1089C00011FA3884C0484E30099032E2012098E70D
:1089D000C148FEF707FA3884C44DC54E21E0B87A85
:1089E000002813D001F049FF069988420ED9059955
:1089F00088420BD201F0FAFD3C73079801F075FF35
:108A0000012001F0C9FF3872BC7211E0B248FEF7D4
:108A1000E9F980B23884B98C884202D38919884236
:108A200006D300210F2001F0C3FE2842B863D6D040
:108A3000B86B411C7ED040047DD58122D20100213B
:108A40000F2002F018F80021102001F0B1FE4106BD
:108A50009D48490E0022503001F0FEFE002001F03A
:108A600065FF002001F017FF974D5035687A072801
:108A7000ABD102229F49681DFCF7B8FB0028A4D1A6
:108A8000284601788F48007881429ED100263546DD
:108A90000AA801F0F8FE04200AAA310E2D020D43A7
:108AA0003102165C0E43401EF7D5BE66FD660026F9
:108AB0003546104601F0D9FE04200AA9320E2D02D7
:108AC000154332020E5C1643401EF7D53E677D67A4
:108AD000B9786A46491CB9707B494D310D791570DA
:108AE000497951700291787B00280AD1012076499A
:108AF00038711288CE310A80787104980575029910
:108B000041757148CE3001886846008803908142E3
:108B10007ED109987849008A08806B4868494C30B2
:108B2000808A48836C48FEF75DF93884788B3A4632
:108B3000FF3001E02CE171E1C33080B26F497883EE
:108B400088420CD94942401850836B486B4B0188CE
:108B50000B33491C89B20180994200D304806849D3
:108B6000032008700998564B81899987C089D88756
:108B7000634BFA6B903B1A601A46B03AD37C1D07E0
:108B80002D0F032D00D07D741A09BA74FC700122D8
:108B9000BA724B4A3E464032118050807879FF21AC
:108BA0009131484357493A6F40180104C8177B6F09
:108BB000891858410206080A104353490790401883
:108BC00006901921079889024018059007984108D6
:108BD0004900080E0902B167F0673B48F36E0A309E
:108BE000B26E01F0ABFF3848736F1630326F01F090
:108BF000A5FF3548F36F1230B26F01F09FFF324D81
:108C0000082068722F48007828707079800000E092
:108C1000C0E0002229461C3001F058FF7079002185
:108C200080001C3001F064FF0120F07224482946C6
:108C3000042251314C30FCF7B5FA31485C3001F078
:108C4000D1FD2F485C30FFF7B1FB1D49803103C9CE
:108C5000FCF760FD404228722748718B05887D2013
:108C6000C0006843401870640B9028480078F07387
:108C700006462748C088FCF710FD03902846FCF7FD
:108C80000CFD0399FCF718FB7F21C905FCF7BBFA23
:108C9000FCF72CFD81B21D480180701E814201D17C
:108CA0000120F872FD8414203E46385EFCF7FCFC7F
:108CB00000910890308CFCF70BFD164A164B2DE006
:108CC000600000200E010020F81100200C0100209F
:108CD000000400502E01002018150020666666660C
:108CE0006666E63F00000840A086010000D0272409
:108CF000983A00003401002040010020E703000002
:108D0000881300205E0B000000AEFCFF2C01002049
:108D1000840D0020F853E3A59B843E40FCF7BCFB88
:108D2000054603910B98FCF7BFFC2A46039BFCF712
:108D3000A5FB009B089AFCF7FDFAFCF7EBFCB0647E
:108D4000BD48008800F0CAFAB07C012871D1122217
:108D5000BA49BB48FCF726FABA4C0822B849A01D0C
:108D6000FCF720FAB64920460A2208313630FCF7D3
:108D700019FAE088B449401E884209D2E08E43289F
:108D800006D2002804D002F037FB642001F0ACFAD0
:108D9000FFF780FDFDF748F8797B3E4688420DD30A
:108DA000012131717179A54A491C717143006A3200
:108DB0000399D15204990D75029A4A75A04A03216C
:108DC0000C3A11540999A14A8B899387C989D18793
:108DD00082009A48F16B9C308150B038C17C737C22
:108DE0000807000F984202D9032800D071749348F5
:108DF000736F643810181630326F01F09FFE70796F
:108E00008E498000002264391C3001F05FFE7079C9
:108E1000002180001C3001F06BFE0AE02A46002190
:108E20000F2001F028FE387B002802D0002001F03E
:108E300032FD388CB98C884200D2C9E5844A891841
:108E40008842FAD88348018888000818F97888424F
:108E500000D27C74804A00210F2001F00CFEB8780B
:108E60007871774800250C380078002812D1F86C0A
:108E7000FDF79EF80646794801883046FCF738F938
:108E80007748761E0088414388B26B490880BE83CC
:108E900000F024FA0020B8737A7B3979521822E066
:108EA000674B0C3B195C00291BD0BC7BAB00641CDE
:108EB000BC73634C9C463C3CE150604B44006A33BD
:108EC0006E001C5B18339C5384001A335C4E1C5993
:108ED00063466C3EF4506D1C33466033491EEDB260
:108EE0001954401CC0B28242DAD8B878032801D2A3
:108EF000B87BB87355490022887B48730490401EA4
:108F000034E000212EE04E4D8B006C3D5E19B446DE
:108F1000EC587668B44223DD484F4D0082377F5BC2
:108F20000997474FA64694003C3F3F590597444F49
:108F30006C3F3C46FE504A3C2C190B9466884A3FD5
:108F40007E533C467A341E193D467A357468EC509F
:108F5000744663465C600B9C099F6780059F776041
:108F6000491CC9B28142CEDB521CD2B28242C8DB5C
:108F70000020364C314D60729C35049A28E02F4910
:108F80002E4E43008231C95A6A36F1528100623650
:108F90007658344F6E50BE4218D0294E3C3E76581B
:108FA000032E13D1677A0626BC467743234E491910
:108FB0005036BE19214F6A37DB191B88B3800B88E6
:108FC000F3804988674631817F1C6772401CC0B2BC
:108FD0009042D4D3194E552050363070AA2070706C
:108FE0000420B070617A06204843811CF170B01CE7
:108FF000FCF7A8FD2083617A062251438A199080EC
:109000003046891D00F038FE164900208200401CC1
:10901000C0B2A9500C28F9D30F4A002180320F208A
:1090200001F029FD01210520002249020007FDF77A
:1090300014FD0DB0F0BD0000160100205C120020F0
:1090400094130020840D0020E7030000600000203E
:10905000983A00001E01002000D027241A010020A9
:1090600018010020FFFF010070470000F0B54A49D9
:1090700085B04848086002F05DF9484800F0EEF815
:10908000474C20834548801C00F0E8F86083434843
:10909000001D00F0E3F8434DA083FF2024302F464D
:1090A000688040373979E1710491E88E3E49C0B259
:1090B00008700390E88F2071A88F6071A87AA07063
:1090C000A8880290A0622889FCF702FB374A384B37
:1090D000FCF7E2F901F0A4F80022364BFCF72AF97C
:1090E000FCF73CFB86B2A681E888019031460090EF
:1090F000FBF7FEFFE08101460298FBF7F9FF7143A1
:109100008EB27D20C00066817043FCF7E1FA2A4AE6
:109110002A4BFCF729FAFCF721FB2082A6827D204E
:10912000C0000099FBF7E4FF6082E083688F207243
:1091300004990120002902D120710A21217201998C
:10914000002901D16421E980039A1749432A01D9F2
:1091500043220A70B98A1A4A914201D90021B98280
:10916000A989494261842084FCF772FEE082228A48
:1091700014491548FDF73AFE14A0A16A00F02AFE32
:10918000E98816A000F026FE298919A000F022FE29
:1091900005B0F0BDC99C00085C000020004F00082D
:1091A0000C010020840D0020160000206666666613
:1091B0006666E63F00000840F853E3A59B843E4006
:1091C00010270000FF7F000018150020B1EAC7A992
:1091D00049443A202564202E0D0A0000CDA8D1B6BE
:1091E000BCE4B8F43A202564206D732E0D0A00000B
:1091F000B5A5B4CECDA8D1B6BBF9D5BECAFDC1BF09
:109200003A202564B8F62E0D0A00000070B586B02D
:1092100014216846FBF7DFFF01250F4EED03002206
:1092200029463046FDF719FC0120002401900294E4
:109230006946009503943046FDF74EFB03200190EC
:1092400002946946009503943046FDF745FB0220E1
:1092500001F04AF806B070BD000400500088704765
:1092600070470000F8B5044600206A461080194D8A
:1092700055222A70AA226A700322AA70661DEE7017
:109280002A716971144A49008918AC712246E81D97
:10929000FBF788FF002007E029186A4689781288C2
:1092A00089186A461180401CB042F5DB611DA81C7C
:1092B000FCF748FC01466846018029190078C8710E
:1092C00068464078087221460931024800F042FBA6
:1092D000F8BD000058140020840D002010B513497B
:1092E0000A8CCB8B9A4201D3D21A0A84104A098C79
:1092F000D2884A437D211018C90048430D490968A6
:10930000401AFCF7D1F90C4A0C4BFCF72DF9FCF78D
:1093100001FA0B49884201DD4A428018002800DA30
:10932000401808490968486110BD00000C01002080
:10933000840D0020A8000020F853E3A59B843E4044
:10934000FF7F000018150020034A1168382389B2F6
:1093500099430143116070470030014010B5FDF79B
:1093600089FB10BD10B59AB034216846FBF733FF76
:1093700014210DA8FBF72FFF1C2112A8FBF72BFFD0
:109380001B4801680324E402A143C2148918016048
:10939000FDF780FD17480169A14301610620009097
:1093A000FF20013002900120039010200490022041
:1093B000099040040B90000100240C900A94684628
:1093C000FDF766FF0F200D9003200E900F94109470
:1093D000012111940DA8FDF749FE81201290032070
:1093E00080041890149412A8FDF78EFD1AB010BDD9
:1093F000007000404010024010480168821511437F
:109400000160C1680E4A1140C16001680D4A1140F7
:109410000160816849084900816001680122920465
:1094200091430160C168FD2212049143C160002193
:10943000016106490448886070470000001002403E
:109440000C40FF88F6FFF6FE0050000800ED00E03B
:1094500070B5026801239B07114C124D984203D04E
:10946000A04201D0A84203D17026B2434E683243D5
:10947000984203D0A04201D0A84204D103231B028A
:109480009A43CB681A4380239A430B691A430260BC
:109490008A68C262096881620121416170BD000071
:1094A000000801400014014010B5CB06DB0E01217D
:1094B000046A99408C430462016A9A401143016234
:1094C00010BD30B58468FF252D021B021343AC4349
:1094D0000B432343836030BD826870239A430A4361
:1094E00007210A438260704730B5026A5208520071
:1094F0000262026A456883697024A3439C080B6872
:10950000A40023430224A2438C6845601443836172
:1095100049684163046230BD30B5026A10239A4342
:109520000262036A4568826973242402A2430C68BC
:1095300024021443202293438A68456012011A438F
:10954000846149688163026230BD30B5026AFF23DD
:1095500001339A430262026A4568C3697024A343D7
:109560009C080B68A400234301246402A2438C6876
:10957000456024021443C3614968C163046230BD7D
:1095800030B5026A01231B039A430262036A4568ED
:10959000C26973242402A2430C68240214430122EA
:1095A000520393438A68456012031A43C4614968B1
:1095B0000164026230BD30B5036A046A6408640065
:1095C00004628469F025AC43120122430A24A343B8
:1095D0000B438261036230BD30B5036A1024A3439C
:1095E00003628469036A0F252D031203AC432243EF
:1095F000A024A343090119438261016230BD000028
:1096000070B501F0E9F80D4C0D4D206502E001F058
:10961000E3F82065A842FAD10020E08220780028F3
:1096200009D0012802D0022805D102E0FCF72CFC69
:1096300001E0FFF73DF900F0C1FF70BD60000020C0
:109640003001CADE10B5818CC90707D001684A68AD
:1096500001235B049A43836A1A434A60818C890719
:1096600007D501684A6801231B049A43C36A1A4359
:109670004A60818C490707D501684A6801239B0429
:109680009A43036B1A434A60818C090707D5016826
:109690004A680123DB039A43436B1A434A60818C77
:1096A000C90607D50268916801231B039943836BA0
:1096B00019439160818C890607D501688A68012366
:1096C0005B039A43C36B1A438A60818C490612D5A7
:1096D00003685A6801210905046C8A4322435A60D1
:1096E000026C8A4207D10268516803235B059943E3
:1096F000436C19435160818C090607D501684A689B
:109700000123DB04806C9A4302434A6010BD0000D1
:10971000F8B500260446C667FDF7A6F90546206899
:109720000068124F000709D501212B460022490588
:109730002046009700F054FA00280DD120680068F8
:1097400040070BD501212B460022890520460097B2
:1097500000F046FA002801D00320F8BD2020606701
:10976000A067603426740020F8BD0000FFFFFF01F1
:10977000F8B5184CC826E078002829D1607900286F
:1097800026D101206071144D686B002700281ED07F
:10979000686BC821081A15E01048E168405C6169EF
:1097A00088470F480A21008848430E490880E0682E
:1097B000401CE060E068C82800DBE760696BC820F7
:1097C000401A761EE168814201D0002EE4DC677108
:1097D000F8BD00004800002000000240BC0C002042
:1097E0001E0100203001002070B5224CE0780028D6
:1097F0003FD1207900283CD1012020711E4EF16913
:1098000000250906002933DA2156625791420AD110
:10981000F06940062CD5A079002829D0A5712089AF
:10982000401C208124E0A179002903D1A0710A20E5
:1098300000F061FD00202056CC2148430F4942181A
:10984000206912181279B262401C00222061A256CF
:10985000CC235A43895881420ADC25612078401C78
:10986000207020780E2800D12570A078401CA070B0
:10987000257170BD4800002000380140940100208F
:1098800010B5806A0022014640314A834A82FEF7C1
:1098900012F910BD70B5846A606FA56F2168896880
:1098A00000260906002906DA212804D15220065391
:1098B000204600F047F820688068400606D5222D33
:1098C00004D15A200653204600F02CF8E06F1021F6
:1098D0000843E0672046FEF7EEF870BD10B501467C
:1098E0000968806A0968890614D400225A210A523C
:1098F00001680A68FF2301339A430A6001688A6895
:10990000520852008A6001688A6840239A438A603C
:1099100020218167FEF76AFA10BD10B5806AFEF754
:1099200066FA10BD01680A68FF2321339A430A6072
:1099300001688A68520852008A60202181670021EC
:109940000166704701680A68C0239A430A602021B3
:109950004167704770B5164CE278002A0CD1227925
:10996000002A09D10122E2700025C82903DC022265
:10997000A256002A01DCE57070BD0123E356CC221B
:1099800053430C4AD1500123E356CC2673439B1812
:109990000A460146181DFBF705FC6078401C607004
:1099A00060780E2800D16570A078401EA070E2E7B4
:1099B0004800002094010020F8B504462669A268FA
:1099C000E76932436669102000253E43236832432D
:1099D00078491E68784F3E4016431E6023685A68D7
:1099E00003263603B243E66832435A602368A2690D
:1099F0008B4201D0266A32439E680B273F02BE434A
:109A000016439E606D4E23686D4AB3420CD1D268F6
:109A10009207920F06D0012A38D0022A34D0032AA6
:109A200020D11EE001201DE0664EB3420AD1D2686B
:109A30000C26324026D0042A28D0082A24D00C2A0A
:109A400010D10EE08B420DD1D6680322920216404F
:109A500018D001229202B61A18D0B61A14D0964223
:109A600000D10820564A0126403A574FF6038B4250
:109A700036D100280CD002280DD0042812D0082896
:109A80001FD11CE00020EDE70220EBE70420E9E70E
:109A9000FDF7A2FB08E01068C00601D5384605E0D6
:109AA0004A4803E0FDF7B8FB002873D06268510014
:109AB0005118814205D81103814202D303E0304698
:109AC000F4E7012566E0010E060250080023301875
:109AD0005941FBF737FB03210902411A3C4A55E083
:109AE000E169B14232D1030000F09BF909070A0D88
:109AF00006250606062B0600E3E7FDF76DFB1CE0D6
:109B0000FDF77AFB19E010686168C00602D54808C5
:109B1000304A01E0304A48088018FBF7E9FA80B281
:109B200001462E4A10399142CBD8511C0140000702
:109B3000400F08432CE0FDF76FFB616840004A08C6
:109B4000EAE76168012248081204E5E7030000F033
:109B500068F909070A0D06260606062C0600B0E776
:109B6000FDF73AFB1DE0FDF747FB1AE0106861685E
:109B7000C00602D54808C01902E014484A08101867
:109B8000FBF7B6FA80B20146144A1039914298D8D0
:109B90002168C8600020206660662846F8BDFDF791
:109BA0003BFB61684A088018EAE761684808801949
:109BB000E6E7000000480040F369FFEF003801408D
:109BC000401002400044004000093D000024F40021
:109BD000FFFC0F0000127A000048E801EFFF0000D0
:109BE000FFB581B017460E4604460A9D09E0681C81
:109BF00007D0FCF739FF0499401AA8420CD8002D71
:109C00000AD02068C1693046884318D00020B84285
:109C1000EDD0002005B0F0BD20680168FF22A13220
:109C200091430160206881684908490081602020D3
:109C30006067A0670020603420740320EAE70120F9
:109C4000E5E7000010B504491020096808620248E1
:109C5000FDF732FF10BD0000DC15002001B5012327
:109C60001A4669460248FEF7C3F80248C06908BDB3
:109C7000DC1500200038014070B50D460646002472
:109C800003E0305DFFF7EAFF641CAC42F9DB70BD16
:109C900001490D20887070474800002010B5074822
:109CA0000A22418A51438184FEF780FCFEF798FD29
:109CB000C82203490348FEF73DF810BD0C010020FF
:109CC000BC0C0020DC150020F8B53D4C00232178A9
:109CD0003C4A1D46082910D0072945D006294ED0F8
:109CE000052950D0042951D0032952D0002954D03D
:109CF000012956D0022958D059E0A17800264A1FE0
:109D000004E0304FBF5DFB189BB2761C9642F8DB37
:109D1000667927799A195118E3786278C9188918F1
:109D2000C9194018C0071AD0012E14D0022E16D11E
:109D300025482449C018FBF735FA01F05DFB642083
:109D400000F0D2FABFF34F8F21492048C860BFF31B
:109D50004F8F00BFFDE759081046FFF783FA2570C3
:109D6000E570A570A571F8BDA1795054491CC8B221
:109D7000A071A178491F8842F5D1082001E06070E8
:109D800007202070F8BDE0700620FAE7607105201A
:109D9000F7E7A070E5700420F3E7552807D101200C
:109DA000EFE7AA2803D10220EBE7032803D02570B0
:109DB000E570A570F8BD032020702071F8BD00008B
:109DC00003010020F4130020840D00200400FA0594
:109DD00000ED00E00FB410B503A9044B044A02984B
:109DE00000F076F910BC08BC04B0184755AB000869
:109DF000500100202021020C01D010211046020A3F
:109E000001D010460839020901D01046091F820806
:109E100001D01046891E420801D0881E7047081ADA
:109E2000704730B47446641E2578641CAB4200D27F
:109E30001D46635D5B00E31830BC1847F8B5044667
:109E40004F1EC8000838211815461E460868496884
:109E50003A4606239A4310D02A463346FBF71CFBAA
:109E60003A46D200083AA3181A687F1E5B68FBF7CF
:109E700061FA06223B469343EED1022F23D0042FF2
:109E800011D0062F2FD12A463346FBF705FBE36A94
:109E9000A26AFBF74FFA2A463346FBF7FDFA636ADC
:109EA000226AFBF747FA2A463346FBF7F5FAE369DD
:109EB000A269FBF73FFA2A463346FBF7EDFA6369DE
:109EC0002269FBF737FA2A463346FBF7E5FAE368DF
:109ED000A268FBF72FFA2A463346FBF7DDFA6368E0
:109EE0002268FBF727FAF8BD002210B5134610468A
:109EF0000149FBF739FB10BD0000F03F10B501220E
:109F0000FBF7AAFB10BD002210B513461046114600
:109F1000FBF72AFB10BD02E008C8121F08C1002A87
:109F2000FAD170477047002001E001C1121F002ADA
:109F3000FBD17047014908607047000054010020C0
:109F400008B50021684601706B46012202212C20D1
:109F500000F0A0FD0221684601706B4601222C2012
:109F600000F098FD08BD000038B504466D20694634
:109F700008706B46012207492E2000F08BFD064930
:109F8000002C01D0054A00E0054A2E2000F068FDB3
:109F900038BD000006080000061800000706000093
:109FA0000716000038B504466B4602220021362011
:109FB00000F036FCB3212300FFF733FF0E0F081526
:109FC0003A3A3A3A1C273A3A2F34483A002168463E
:109FD000017040784108490014E06946087880081B
:109FE0008000401C04E06946087880088000801CDE
:109FF00008701DE0684602780A40483202704178D5
:10A00000802001436846417012E0684602780A40A9
:10A01000027040784106490EF4E76946487802210B
:10A02000084303E069464878FD21084069464870C6
:10A030006B4601220021362000F02CFD012200ABEE
:10A0400011463620013300F025FD38BD69460878F9
:10A05000CF21084069462030CAE708B50321684689
:10A060004170012101706B4602220021362000F070
:10A0700011FD0122D20306212D2000F0F1FC012068
:10A0800000F032F90120FFF78DFF08BD08B5020A84
:10A0900069464A7008706B46022204212D2000F0A8
:10A0A000F9FC0320694608706B46012206212D2029
:10A0B00000F0F0FC0020694608706B460122062182
:10A0C0002D2000F0E7FC0A212D2000F071FB08BDD7
:10A0D000FFB58DB00446002506E025280AD0109A69
:10A0E0000F999047641C6D1C20780028F5D12846F4
:10A0F00011B0F0BD00270121484A009700E0074356
:10A10000641C23780846203B98401042F7D1207801
:10A110002E2817D1042007436078641C2A280CD10C
:10A120000E98641C02C800910E900BE000990A2260
:10A13000514330394018641C009020780146303972
:10A140000929F3D920780028D1D0642808D06928BB
:10A1500006D075281ED0109A0F9990476D1C5BE0B1
:10A160000A200E99019001C90E91002802DA40429E
:10A170002D2102E0390504D52B216A4611720121F7
:10A1800003E0F90704D02021F7E70BAE0B910DE0B7
:10A190000021FAE70A200E99019001C90E91F7E714
:10A1A0000199FAF7A5FF3031761E31700028F7D1FA
:10A1B00003A8801B20300190780701D5009801E0AA
:10A1C000012000900199884201DD401A00E0002042
:10A1D0000027009006E002A8109AC05D0F999047F2
:10A1E0006D1C7F1C0B988742F5DB04E0109A302031
:10A1F0000F9990476D1C0099481E00900029F5DCCE
:10A2000005E03078109A761C0F9990476D1C0199E3
:10A21000481E01900029F4DC641C65E70928010050
:10A22000F8B54A002B4B520DD6182B4A0C46054662
:10A23000142E2BDA002E12DA284BFBF77BF80022C3
:10A240001346FBF7CBFB40D2002C03DA0124E407D2
:10A2500000253AE02046284337D0214C14E0214F16
:10A260000B46F7403B402B4331D01C4BFBF762F8C9
:10A2700000221346FBF7B2FB27D2002C03DD01209E
:10A280000005F0400419BC4300251EE0332E1EDCFF
:10A2900033460027143BFF43DF40384217D00F4BB3
:10A2A000FBF7F2F800221346FBF798FB0DD2002CC7
:10A2B0000ADD142E0CD03420811B01208840401967
:10A2C000A84200D2641C0546BD4321462846F8BD7D
:10A2D000641CF9E701FCFFFF9C7500883CE4377EB5
:10A2E0000000F03FFFFF0F007D2110B5C90048437B
:10A2F00000F001F810BD002140E000BF00BF00BF2A
:10A3000000BF00BF00BF00BF00BF00BF00BF00BF55
:10A3100000BF00BF00BF00BF00BF00BF00BF00BF45
:10A3200000BF00BF00BF00BF00BF00BF00BF00BF35
:10A3300000BF00BF00BF00BF00BF00BF00BF00BF25
:10A3400000BF00BF00BF00BF00BF00BF00BF00BF15
:10A3500000BF00BF00BF00BF00BF00BF00BF00BF05
:10A3600000BF00BF00BF00BF00BF00BF00BF00BFF5
:10A3700000BF00BF00BF00BF00BF491C8142BCD36B
:10A3800070470000FEB504460020019000906079FF
:10A39000734940000E5A61782578491E7148CFB242
:10A3A0000163042D77D0072D75D00021029121780B
:10A3B00001736C49E379012292058969002B6CD005
:10A3C000914381616748217A4173217A82698907C3
:10A3D000890B0A4382610021042000F04CFB3246C5
:10A3E00061492E2000F03CFB3846FFF7BDFD5F4E73
:10A3F0000522705D810040185D49431807212B201C
:10A4000000F048FB5B49029801220B180B21282021
:10A4100000F040FB705D584980000A580C2128204C
:10A4200000F029FBE079554980004018A1794900E6
:10A43000425A0221272000F013FB51487E00825B24
:10A440000421272000F00CFBE079002829D0A07817
:10A4500004282CD0282069460872202206212720B3
:10A4600000F0FEFA02AB01222621272000F012FBA9
:10A47000444938014018E1788900425808212720D2
:10A4800000F0F9FAA17A601C627A0902114313D034
:10A4900016E000E001E0012188E71143F608816140
:10A4A00090E764220621272000F0DAFAE0E7102086
:10A4B000694608720246D1E733490172090A4172BE
:10A4C000417A007A0A0202432021272000F0C8FACC
:10A4D0002E4F0C2123203A6800F0CDFAF019828823
:10A4E0000421232000F0BCFAA07900280BD0E079E9
:10A4F0002749012243180021212000F0CBFA032034
:10A500000190012000902A07120F10010243607889
:10A5100000218007000B02430198000502430098C8
:10A52000400402432079C006400902436079C00616
:10A5300002431F2000F09FFAA078617801230843AE
:10A5400002040848DB030261E179490319430A4325
:10A5500002610021082000F08EFA0020FEBD0000FC
:10A56000D0B40008580100200428000078B4000886
:10A57000170000203500002080B40008A0B40008B7
:10A58000ACB40008B0B400084110000098B4000852
:10A590003700002038B50C4607498A8B002102435A
:10A5A0002C2000F05DFA684604706B4601220621FB
:10A5B0002C2000F06FFA38BD5801002010B5FFF7CD
:10A5C000BFFC10BD10B504460421362000F0F0F8A1
:10A5D0000121C902002C01D0084300E08843024653
:10A5E0000421362000F047FA10BD000038B54020A5
:10A5F0006946087000210E2000F0DAF804460022B7
:10A6000011460E2000F037FA6B46012200210D2082
:10A6100000F040FA074A00210F2000F02CFA00F069
:10A6200005FA224600210E2000F025FA02480021FA
:10A63000017338BDF8FF2724780100207CB505465A
:10A640000420694608704B4C00206075214620317B
:10A65000206348710873A0836063A06300F0BCF8B6
:10A66000454E206002E000F0B7F82060B042FAD119
:10A670000020FFF797FC41480078242801D92438AE
:10A6800006E00621FAF734FD0622101A40010843BD
:10A69000020601040A4301020A43024300211E206C
:10A6A00000F0E9F96B4601220021242000F0F2F9C4
:10A6B0001E20FFF7EBFC86B2300AA0730420FFF7E0
:10A6C000E5FC0006000E0DD002206946087101ABC2
:10A6D000012212212D2000F0DDF9A08B01210903B8
:10A6E0000843A08300F078F820600620FFF7CEFC36
:10A6F00060600720FFF7CAFCA060F006C00E20755E
:10A7000001D110202075C0B200F000FAE80707D090
:10A71000FFF7A3FCA08B0121C9020843A0830AE034
:10A720000521362000F02EF8154908400246052183
:10A73000362000F095F90120FFF734FC00210420B9
:10A7400000F036F8A0610021262000F031F8152134
:10A750008903084302460021262000F08CF90022DC
:10A760002621362000F07CF900F036F82060002029
:10A770007CBD0000580100203001CADE1600002018
:10A78000FFFD000038B5094C89B280B26B46022249
:10A7900000F046F8002806D1684640780102684675
:10A7A0000078081884B2204638BD0000FFFF000082
:10A7B00038B50024E44389B280B26B46042200F02D
:10A7C0002FF8002806D103216846435C2202D418E2
:10A7D000491EFAD5204638BD10B500210846FFF7BE
:10A7E000E7FF10BD10B5044605211520FFF7CAFF8D
:10A7F000E08100212E20FFF7C5FF2080231D0822C5
:10A800000021122000F00CF807211520FFF7BAFFF5
:10A81000608000211020FFF7CBFF000DA08110BD4C
:10A8200038B5002909D0402420436C462070C8B2B6
:10A830007F2906D8607002200AE06946087001206E
:10A8400006E0802420436C466070C809A070032095
:10A85000694600F0ABFD38BD10B5144603460A4604
:10A8600021461120FFF7DCFF10BD10B5034605227D
:10A8700000211520FFF7D4FF10BD10B501210620DF
:10A88000FFF796FF10BD10B50346052200211720E3
:10A89000FFF7C6FF10BD38B50546002069460870B1
:10A8A00000F0C4F8FF2401342246002D01D0032219
:10A8B000120200210D2000F0D3F8002D13D06B46BA
:10A8C000012203210F20FFF7ABFF68460078000745
:10A8D00009D5FFF78BFE224600210D2000F0C0F8BD
:10A8E0000020C04338BD002038BD10B5024601210C
:10A8F0000A2000F0C0F810BD10B5044600211A204F
:10A90000FFF756FF000D22030005120B0243002142
:10A910001A2000F0B0F810BD10B5024602492E20F2
:10A9200000F09EF810BD000004180000F8B50546C0
:10A930006B46012203210420FFF772FF0126114C10
:10A940003607002D0DD02A4600210C2000F088F893
:10A95000694608781021084369460870A0693043A9
:10A9600007E069460878EF21084069460870A06949
:10A97000B0430B46A06101220321042000F08AF8B5
:10A98000F8BD00005801002010B502460021182033
:10A9900000F066F810BD0000F8B5074600256846CF
:10A9A0000570B807204C2E4600280ADA8020694638
:10A9B00008706B46012200210D2000F06BF8012089
:10A9C0002073F8076946087821D0062108436946B4
:10A9D00008706B46012200210D2000F05BF8032176
:10A9E0000F20FFF7CFFE8121C900084219D0402077
:10A9F000694608706B46012200210D2000F04AF8DC
:10AA00000020FFF7DFFD00252673ED4309E002215A
:10AA10000843694608706B46012200210D2000F0B2
:10AA200039F82846F8BD0000780100201CB56B46B7
:10AA3000012203210F20FFF7F3FE68460078402231
:10AA4000C1091040C9014000814208D00120694677
:10AA50000871024601AB03210D2000F01BF81CBD5C
:10AA600008B56B461A70120A5A7089B280B2022277
:10AA700000F010F808BD38B500236C46E254120A05
:10AA80005B1C042BFADB89B280B22346042200F05F
:10AA900001F838BD38B58024002909D0C0252843E5
:10AAA0006D462870C8B27F2907D86870022009E077
:10AAB000204369460870012004E020436870C809FB
:10AAC000A8700320694600F0B3FC38BD10B51446E9
:10AAD000012312189B029A4202D90020C04310BDE4
:10AAE0000B46821E21460920FFF7D4FF002010BD2F
:10AAF00010B5054A8905126901430A43002108205F
:10AB0000FFF7B9FF002010BD5801002038B50446FA
:10AB10006B4601220E212B20FFF782FE684600784B
:10AB2000E10640094001C90E0143684601706B46C9
:10AB300001220E212B20FFF7ADFF38BD10B50021FB
:10AB400042541C06120A22431B0A491C0429F7DB43
:10AB500010BD000013B501231A4669460248FDF7EF
:10AB600047F900981CBD0000DC150020F0B5C54A6F
:10AB700000248FB091420ADA4B005B08934206D85A
:10AB800001254A006D05EA4205D1002803D0FFF7F0
:10AB9000B5F90FB0F0BD01252D05A94219DA03431F
:10ABA00008D0002910DA0120FFF7C4F9FFF7ABF94C
:10ABB0000FB0F0BD0220FFF7BDF9FFF795F90122B4
:10ABC000D20751400FB0F0BD3524E4433622FAF7E6
:10ABD00043FD0A15AC4B1219D4180A03120BAB49EA
:10ABE000AB4B56182E403146594011430192321555
:10ABF00012190B920022FAF741FC019A0446921CAA
:10AC00001003A44E000B0D467E44032860D220465C
:10AC100073683268FAF7CEFE1CD10B98002815D065
:10AC2000FAF742FD04460E469B4A9C4BFAF734FC69
:10AC30000D4607469A4A9B4B20463146FAF72CFCB4
:10AC40003A462B46FAF776FB0FB0F0BD71683068D4
:10AC50000FB0F0BD944A954B20462946FAF71CFCEC
:10AC60000022934BFAF710FC06460F4622462B466D
:10AC700010461946FAF710FC32463B46FAF70CFC30
:10AC800006460B980F4600281DD0FAF70DFD824AA4
:10AC9000824B05910490FAF7FFFB32463B46FAF7E8
:10ACA000F3FB22462B46FAF7E9FB04460D467C4AA5
:10ACB0007C4B05990498FAF7EFFB22462B46FAF7EE
:10ACC000DDFB0FB0F0BD0B46324620462946C4E0FE
:10ACD000012300229B072046FAF72CFB02460B4675
:10ACE00020462946FAF740FC06460F460B98FAF72D
:10ACF000DBFC32463B460591049010461946FAF7B4
:10AD0000CBFB09910C906B490198099B421800926A
:10AD10000C9A19461046FAF7BFFB024607910A90B3
:10AD2000654901980B1A6548019303217844079BF4
:10AD3000FFF784F8079B0A9AFAF7AEFB0E905F487C
:10AD40000D9104217844079B0A9AFFF777F8099B35
:10AD50000C9AFAF7A1FB019B009A1A4300920D9BF3
:10AD60000E9AFAF7E7FA009A01910C90002A4DDD4D
:10AD70000022D24320462946FAF76EFC22462B4693
:10AD8000FAF78AFB00910A900B9800282BD0424AD0
:10AD9000424B05990498FAF77FFB07910E90019BAF
:10ADA0000C9A00990A98FAF7C5FA32463B46FAF728
:10ADB00073FB079B0E9AFAF7BDFA009B0A9AFAF703
:10ADC00063FB22462B46FAF759FB04460D46344AEC
:10ADD000344B05990498FAF75FFB22462B46FAF7A5
:10ADE0004DFB0FB0F0BD019B0C9A0A98FAF7A2FA3E
:10ADF00032463B46FAF750FB009B0A9AFAF744FBAF
:10AE000022462B46FAF740FB0FB0F0BD0B98002806
:10AE100027D0214A214B05990498FAF73DFB079169
:10AE2000009020462946019B0C9AFAF727FB3246F0
:10AE30003B46FAF731FB079B009AFAF71FFB2246C5
:10AE40002B46FAF71BFB04460D46154A154B059990
:10AE50000498FAF721FB22462B46FAF70FFB0FB0B6
:10AE6000F0BD0B46204629460C9AFAF707FB3246FE
:10AE70003B46FAF711FB22462B46FAF705FB0FB0CB
:10AE8000F0BD00000000F07F01FCFFFF645F0900DF
:10AE90000000F03F54090000763C7935EF39EA3D77
:10AEA0000000E0FE422EE63F555555555555D53F1D
:10AEB0000000E03F86EBF9FF51B80600F8070000FC
:10AEC000F8B504463048002581420ADA4A005208A3
:10AED000824206D8012348005B05D84205D1002CE8
:10AEE00003D02046FFF70AF8F8BD01231B0599425D
:10AEF00019DA224307D000290EDA0120FFF71AF8E9
:10AF0000FFF701F8F8BD0220FFF714F8FEF7ECFF99
:10AF10000122D2075140F8BD3525ED4336222046A7
:10AF2000FAF79AFB044608154019184A0D038018D1
:10AF3000C20F17492D0B891A09050D438018FAF71E
:10AF4000B3FB06460F4620462946FFF70FFE114A7F
:10AF5000114BFAF7A1FA04460D46104A104B304641
:10AF60003946FAF799FA22462B46FAF7E3F90D46E5
:10AF700004460C4A0C4B30463946FAF78DFA224605
:10AF80002B46FAF7D7F9F8BD0000F07F01FCFFFF70
:10AF9000FF0300000EE526157BCBDB3F362BF111BE
:10AFA000F3FE593D00609F501344D33FFBF76AFD09
:10AFB000FEF7D8F9FDF70EFB41494248002522C0B3
:10AFC00005608561C56140490562C1600838FBF7CD
:10AFD0008FFEFDF7EBFAFDF703FCFDF79FFBFDF796
:10AFE000B1FA052601223607D1033046FBF735FDBD
:10AFF000FEF73CF8FAF788FDFAF7FAFDFAF7D2FD0A
:10B00000FCF766FF0721B015FFF7C4FAFFF7D6FA81
:10B010002E4C0A21608A01224843A0841103304645
:10B02000FBF71BFD2748C8222949C430FCF782FEE4
:10B03000284F294EE07800283FD0E07900283CD006
:10B04000FEF790F9E570FAF7EBFF20700F280AD9A8
:10B05000012211033046FBF700FDFEF7D1FA002272
:10B060000121090309E0012251033046FBF7F5FCF9
:10B07000FEF7C6FA0022012149033046FBF7EDFC3A
:10B08000FDF74AF8A08C002801D0401EA084134888
:10B09000A18C00780843CDD13878002801D003284E
:10B0A000C8D10121C9023046FBF7D2FC0028C1D12A
:10B0B00001210846FBF70EFFBCE7FDF72DF8B9E7C5
:10B0C000007C004018150020FFFF00000C0100204C
:10B0D000BC0C002071000020000400504E00002035
:10B0E00010B586B01748FBF788FD14216846FAF7BB
:10B0F00072F815480090032001900020029005206E
:10B1000069460007FBF7E8FB69461048FBF7E4FBDC
:10B1100069460F48FBF7E0FB01210846FBF7DAFE22
:10B12000FF2401342046FBF7ADFE0A4908680422DB
:10B13000104308602046FBF7B5FEFBF7BBFE06B0E8
:10B1400010BD000018150020FFFF00000004005093
:10B15000000800500070004010B50446FCF778FF6E
:10B160004E20FCF748FFFCF7ACFFE0B2FCF743FFD2
:10B17000FCF7A7FFFCF76CFF4F20FCF73CFFFCF748
:10B18000A0FF0020FCF70AFF0446FCF77CFF2046E6
:10B1900010BD70B50D460446FCF75AFF4E20FCF773
:10B1A0002AFFFCF78EFFE0B2FCF725FFFCF789FFD2
:10B1B0002846FCF720FFFCF784FFFCF764FF0A2019
:10B1C000FFF799F870BD000010B52421002000F0B1
:10B1D0004DF81B48FFF78FF800210F2000F046F8CC
:10B1E0000521102000F042F80421112000F03EF863
:10B1F00083217F2000F03AF869217F2000F036F8A3
:10B20000BD217F2000F032F80E480078262804D1B6
:10B21000002240218C2000F019F8012000F02AF8CB
:10B22000094814210187282000F020F80A20FFF7A0
:10B2300062F8012000F036F8012000F043F810BD5C
:10B24000204E000000000020840D0020F8B51746B5
:10B250000E4605460024FFF77FFF3946B4433140D0
:10B260002143284600F002F80020F8BD10B5FFF792
:10B2700090FF10BD10B500280AD000212720FFF74D
:10B28000F5FF04211920FFF7F1FF8721162005E0C3
:10B2900000211620FFF7EAFF00211920FFF7E6FF43
:10B2A00010BD000010B5002801D0002200E080226F
:10B2B00080211120FFF7CAFF0148FFF71CF810BDDD
:10B2C000A086010010B5002811D001212F20FFF722
:10B2D000CDFF62213020FFF7C9FF46213120FFF763
:10B2E000C5FF32210846FFF7C1FFA22100E022215D
:10B2F0003320FFF7BBFF10BD0C480D4A0188914277
:10B3000010D1C18832290DD3C18E43290AD8818F2B
:10B31000012907D8C08F012804D80448403080880C
:10B32000012801D90120704700207047840D0020BA
:10B33000AA55000010B50122920219491948FAF7DE
:10B34000CDFC1748184902888A4227D00180042181
:10B350008180FF21F531C1800A21018100211E2257
:10B360004181D24382810122C281018401824182D2
:10B370008182C182018381834323C38602230387A1
:10B38000782343878287C287024640329182918028
:10B39000118451849184C18300F02EF810BD000007
:10B3A000840D002000FC0008AA550000F0B58C4672
:10B3B00000251026052109078E620E4C08E067461D
:10B3C0007F5DE760A768FF07FCD0E7681F706D1C12
:10B3D0008542F4DB0020074606E0E760A568ED073C
:10B3E000FCD0E5681D54401C9042F6D38E610020CD
:10B3F000F0BD00000030014070B5FFF77DFF002870
:10B4000001D0012070BD72B60124074DA40221466F
:10B410002846FAF749FC002804D02246034928466A
:10B42000FAF7E6FC62B670BD00FC0008840D00204F
:10B43000F0B50025102605279C463F070B46BE6247
:10B440000C4C06E0595DE160A168C907FCD0E168D9
:10B450006D1C8542F6DB002007E06146095CE16077
:10B46000A168C907FCD0E168401C9042F5D3BE61D9
:10B470000020F0BD0030014000000102030400057F
:10B48000405C0000A05C0400C06C0800805C04000C
:10B49000E03F1E00E07D1E0007A9022570889B8802
:10B4A0000A001600010006000100020087008D005E
:10B4B0002D001A3152001A339A001A351D011A371D
:10B4C0006B003B31BE003B335E013B3596023B37A0
:10B4D000000099599959EB518F421E45142E008056
:10B4E000EB51F5283333E13A703DE13AC235852B13
:10B4F000C2353333C235C235AE47E13A5138A33095
:10B50000513800000000000000000102030406079B
:10B510000809030406080C10182030000000000180
:10B52000020304000000000004FA97999999D93F9A
:10B53000AF788E1DC571CC3F9FC678D0099AC33FA6
:10B54000935555555555E53F599322942449D23F7B
:10B55000DE03CB966446C73F44523EDF12F1C23F42
:10B56000000000000000000088B500080000002076
:10B5700058010000285A0008D4B5000858010020DE
:10B58000B0190000269F0008021627130704380D83
:10B59000091E080540082609104008560A131D0414
:10B5A0003B08BE0526D8BC4010085201031CC84207
:10B5B0004924E103498C0A000A30418FC2F5285C16
:10B5C0006F5E401402021415090901020A1881A8CD
:04B5D0000132922092
:04000005080050C1DE
:00000001FF
